:020000040000FA
:100000008501860183161C308500803086008101C1
:1000100083120B118C01AD01143093008A019021E1
:10002000051E74280A301A20900003011A2091003E
:100030000C14272882077E3448343D346D344B3409
:10004000673473344C347F344F3400343634810198
:100050000B1100000B1D29280B11D13081008C1BC6
:10006000C328930B362814309300D620AC0803190C
:100070003B28AC032928051E4B28AD1C4328AD1096
:100080006430AC002928861F67282D1C29282D10D4
:100090006430AC002928AD182928AD146430AC00B8
:1000A00000307C21AA3A03195A28013090009100AF
:1000B0000C14292801307C21553A031D55280230A3
:1000C0007C21900003307C2191000C1429282D18EC
:1000D00029282D146430AC008C1B72288C178601E3
:1000E0000C1129288C13292890219021051E742891
:1000F00090219021E7308C05051983288C1103018C
:100100001A20900087288C1501301A20900085193C
:100110008E280C1203011A20910092280C1601302F
:100120001A2091000C1481010B1100000B1D952861
:100130000B11D1308100930B952814309300D620F9
:100140000519AA288C1DB1288C110B301A2090009B
:100150000C14B1288C19B1288C1505301A20900088
:100160000C148519BB280C1E95280C120B301A2074
:1001700091000C1495280C1A95280C1605301A209D
:1001800091000C1495280C19CC28051929280C1558
:10019000A101A201A3012928A30FD128A20FD128D0
:1001A000A10A85192928F3208C1329280C1CDD2885
:1001B00010088D0011088E000C108C18E9288C1482
:1001C0008501000000000D08860000000000851475
:1001D00008008C108501000000000E088600000059
:1001E00000000514080001309400193095004030DB
:1001F00096002108970022089800230899004621BC
:100200001508A4001608A5002321290E0F3903198B
:100210000A3E1A20900088000230890082212908B5
:100220000F391A2091008800033089008221AA30FA
:100230008800003089008221553088000130890013
:1002400082210C14080003101030A000AB01A8019B
:10025000A901A50DA40DA90DA80DAB0DA00B312969
:100260000800293084003B21283084003B212B30BA
:1002700084003B21292903300007AA00AA19800025
:1002800030300007AA00AA1B800008001830A00028
:1002900014089D0015089E0016089F009401950102
:1002A00096019A019B019C0103109F0D9E0D9D0DCF
:1002B0009C0D9B0D9A0D17081A02031D652918083D
:1002C0001B02031D652919081C02031C7629190845
:1002D0009C02031C9B031B08FF3A03199A0318088E
:1002E0009B02031C9A0317089A020314960D950D9E
:1002F000940DA00B5429080089008316081483125A
:1003000008080800831608120815000055308900F7
:10031000AA3089008814081E8B290811831208004E
:0A032000A0010000A00B91290800C5
:00000001FF
